:020000040800F2
:1000000000060020E1010008CD0D0008D10D000818
:10001000250E0008D10D0008F90D0008E3010008C5
:10002000E3010008E3010008E3010008892E00084D
:10003000E3010008E3010008E3010008E301000810
:10004000E3010008E3010008E3010008E301000800
:10005000E3010008E3010008E93000081531000859
:10006000413100086D31000899310008E3010008B2
:10007000E3010008E3010008E3010008E3010008D0
:10008000E3010008E3010008E3010008E3010008C0
:10009000E3010008E3010008E3010008C53100089E
:1000A000E3010008E3010008E3010008E3010008A0
:1000B000052F0008E3010008E3010008E301000840
:1000C000E3010008E3010008E3010008E301000880
:1000D000E3010008E3010008E3010008E301000870
:1000E0002D320008E3010008E3010008E3010008E5
:1000F000E3010008E3010008E3010008E301000850
:10010000E3010008E3010008E3010008E30100083F
:10011000E3010008E3010008E3010008E30100082F
:10012000E3010008E3010008E3010008E30100081F
:10013000E3010008E3010008E3010008E30100080F
:10014000E3010008E3010008E301000809270008B3
:10015000E3010008E3010008E3010008E3010008EF
:10016000E3010008E3010008E3010008E3010008DF
:10017000E3010008E3010008E3010008E3010008CF
:10018000E3010008E3010008E3010008E3010008BF
:10019000E3010008E3010008E3010008E3010008AF
:1001A000E3010008E3010008E3010008E30100089F
:1001B000E3010008E3010008E3010008E30100088F
:1001C000E3010008E3010008E3010008E30100087F
:1001D000E3010008E3010008E3010008E30100086F
:1001E00002E000F000F8FEE772B6394880F30888B4
:1001F000384880F3098838484EF60851CEF200019D
:10020000086040F20000CCF200004EF63471CEF2ED
:1002100000010860BFF34F8FBFF36F8F40F2000003
:10022000C0F2F0004EF68851CEF200010860BFF334
:100230004F8FBFF36F8F4FF00000E1EE100A4EF6C4
:100240003C71CEF200010860062080F31488BFF3F1
:100250006F8F01F02BFF02F0B5FD4FF055301F49B5
:100260001B4A91423CBF41F8040BFAE71C49194A6A
:1002700091423CBF41F8040BFAE71A491A4A1B4B5A
:100280009A423EBF51F8040B42F8040BF8E70020F5
:100290001749184A91423CBF41F8040BFAE701F0B4
:1002A00009FF02F0E3FD144C144DAC4203DA54F89C
:1002B000041B8847F9E700F03FF8114C114DAC42A0
:1002C00003DA54F8041B8847F9E701F0F1BE000097
:1002D000000600200026002000000008000000208A
:1002E00000060020383600080026002028260020BE
:1002F0002826002014320020E0010008E001000858
:10030000E0010008E00100082DE9F04F2DED108A12
:10031000C1F80CD0C3689D46BDEC108ABDE8F08FD3
:10032000002383F311882846A047002001F048FBF2
:1003300001F07EFA00DFFEE71B4B6FF0040270B5A0
:100340001A70032200245A700F229C70DC701C71FA
:100350005C719C71DC711C725C729A72DC7201F0CF
:1003600077FE064601F09CFE054650B90F4B9E42B3
:1003700017D001339E4241F2883412BF0546002453
:100380000125002001F06EFE0DB100F057F800F0DD
:10039000F3FC00F083FB204600F0A8F800F04EF8D4
:1003A000F9E70446EDE700BF28260020010007B06A
:1003B00008B500F011FBA0F120035842584108BDD8
:1003C00007B541F21203022101A8ADF8043000F094
:1003D00055FB03B05DF804FB10B5202383F31188AF
:1003E0001248C3680BB101F06FFB114A0F4800239C
:1003F0004FF47A7101F02EFB002383F311880D4C2A
:10040000236813B12368013B2360636813B16368F9
:10041000013B6360084B1B7833B9636823B9022042
:1004200000F024FC3223636010BD00BF342600209E
:10043000D90300085027002048260020254B264AD3
:1004400010B51C461968013142D004339342F9D1EA
:100450006268224B9A423BD9214B9B6803F10063AF
:1004600003F580339A4233D2002000F031FB1D4B5C
:100470000220187000F0F2FB1B4B1A6C00221A6469
:10048000196E1A66196E596C5A64596E5A665A6E0C
:100490005A6942F080025A615A6922F080025A6118
:1004A0005A691A6942F000521A611A6922F0005220
:1004B0001A611B6972B64FF0E0232021C3F8084D82
:1004C000D4E9003281F311889D4683F308881047F0
:1004D00010BD00BF0000010820000108FFFF000858
:1004E0002826002048260020003802402DE9F04F41
:1004F00093B0DFF8E0B200902022FF210AA8DBF8D9
:10050000087000F0E3FBAE4A1378A3B9AD480121AF
:10051000C3601170202383F31188C3680BB101F00D
:10052000D3FAA94AA74800234FF47A7101F092FA4E
:10053000002383F31188009B13B1A44B009A1A6027
:10054000A34A009E00231370A04A994653601D469B
:100550001C469846012000F081FB26B19B4B1B688E
:10056000002B00F00082002000F036FA0390039B7D
:10057000002BF2DB012000F067FB039B213B122BD9
:10058000E8D801A252F823F0D5050008FD050008BF
:100590006B060008550500085505000855050008BC
:1005A000FF060008D3080008E50700084F08000808
:1005B000770800089D08000855050008AF080008E6
:1005C0005505000825090008ED0600085505000836
:1005D0006D0900080220FFF7EBFE002840F0ED81D6
:1005E000009BB9F1000F08BF1E4641F212330221F1
:1005F00005A8ADF8143000F041FAABE74FF47A707B
:1006000000F0EAF9031E0193EADB0220FFF7D0FEB7
:1006100082460028E4D0019B581E042800F2CF81B6
:10062000DFE800F0030D10131600052305930421E5
:1006300005A800F023FA55464FF0000856E065483B
:100640000421F6E764480421F3E764480421F0E755
:100650001C25284600F03EFA04350590042105A823
:1006600000F00CFA2C2DF4D1E5E7002CB8D0002DC9
:10067000B6D00220FFF79CFE0446002800F0A281BD
:10068000012000F025FA524B0220187000F0E6FA23
:1006900000255FFA85F9484600F02AFA064658B167
:1006A000484600F035FA01350028F2D12546A1462A
:1006B000064641F212139AE7454A012302201370BD
:1006C00000F0C2FA3746DBF80830BB4207D938469B
:1006D00000F000FA013040F077810437F3E73C4B3B
:1006E00000271F70394BA1465F60254600F03AFB9A
:1006F00014B1002D18BF0026FFF762FE2AE7002C78
:100700003FF46EAF002D3FF46BAF314B02201870F9
:1007100000F0A4FA322000F05FF9B0F1000AC0F254
:1007200051811AF0030440F04D81DBF808200AEBF8
:100730000703934200F24681BAF5807F00F34281BD
:10074000274B0193A2450EDD4FF47A7000F044F977
:100750000390039A002AC0F23581019B039A03F8A3
:10076000012B0134EDE7C820FFF722FE04460028E4
:1007700000F028811F2F11D8C7F1200252450AAB83
:1007800027F0030028BF524615490192184400F093
:1007900077FA019A1248FF2100F098FA4FEAAA036B
:1007A0000F490193CAF38702384600F097FA0546CD
:1007B000002800F00C81019B044607EB830795E7B6
:1007C0004C27002034260020D903000850270020A1
:1007D00048260020282600202C2600203026002035
:1007E0004C2600200220FFF7E3FD00283FF4F8AE7E
:1007F00000F0B8F900283FF4F3AE4FF0000A53467A
:10080000DBF8082052451CD9BAF11F0F12D80A9AFA
:1008100001320FD02AF0030212A90A4452F8202C08
:1008200005921846042205A900F010FB0AF1040AFB
:100830000346E5E75046019300F04CF9019B059013
:10084000EFE70593042105A800F018F94EE700230F
:10085000642104A8049300F0EBF800287FF4C0AEF4
:100860000220FFF7A5FD00283FF4BAAE049800F07F
:1008700061F90590E6E70023642104A8049300F0E1
:10088000D7F800287FF4ACAE0220FFF791FD0028D6
:100890003FF4A6AE049800F05DF9EAE70220FFF706
:1008A00087FD00283FF49CAE00F06CF9E1E70220E0
:1008B000FFF77EFD00283FF493AE05A9142000F059
:1008C00067F904218246049004A800F0D7F8514645
:1008D000B9E7322000F080F8B0F1000AFFF680AEF0
:1008E0001AF0030F7FF47CAEDBF808200AEB080354
:1008F00093423FF675AE0220FFF75AFD00283FF401
:100900006FAE2AF0030AC244D0453FF4EFAE404632
:1009100000F0E0F80421059005A800F0AFF808F118
:100920000408F1E74FF47A70FFF742FD00283FF426
:1009300057AE00F017F900283FF4BBAE0A9B013315
:100940000CD008220AA9002000F0C8F900283FF4C2
:10095000B0AE2022FF210AA800F0B8F9FFF730FD61
:100960001C4801F033F813B0BDE8F08F002C3FF4C1
:1009700037AE002D3FF434AE0023642105A8059363
:1009800000F056F8824600287FF42AAE0220FFF7D6
:100990000FFD019000283FF423AEFFF711FD41F257
:1009A000883001F013F8059800F00EFA00F0DAF93B
:1009B000019B56461D461C46CCE5044696E64FF084
:1009C00000080DE62C460BE62546A14671E62546B5
:1009D0006FE600BFA086010073B5124B1B78013390
:1009E000DBB20024012B8DF8074013D80E4D2A6886
:1009F0004FF47A73166A0DF10701A0FB033201224E
:100A00002846B047012805D1084B9DF807001C7007
:100A100002B070BD4FF4FA7000F0D8FF4FF0FF3015
:100A2000F6E700BF00260020402A0020842700208F
:100A300038B50F4B1B780133DBB2012B10D80D4CAE
:100A400022684FF47A73156AA1FB0332014604222F
:100A50002046A847042803D1074B0020187038BD52
:100A60004FF4FA7000F0B2FF4FF0FF30F7E700BF2D
:100A700000260020402A00208427002030B4054CA6
:100A80002368DD69044B0A46AC460146204630BC6B
:100A9000604700BF402A0020A086010070B501F029
:100AA000DDF9094E094D30700024286833788342FF
:100AB00008D901F0CDF92B6804440133B4F5803F27
:100AC0002B60F2D370BD00BF85270020582700207F
:100AD00001F072BA00F1006000F5803000687047E4
:100AE00000F10060920000F5803001F0FDB90000D7
:100AF000054B1A68054B1B789B1A834202D9104498
:100B000001F0A6B900207047582700208527002053
:100B100038B5074D04462868204401F0A1F928B9EA
:100B200028682044BDE8384001F0B2B938BD00BFA4
:100B30005827002010F003030AD1B0F5007F05D834
:100B400000F10050A0F51040D0F80038184670476A
:100B50000023FBE700F10050A0F51040D0F8100A88
:100B600070470000064991F8243033B10023086A29
:100B700081F824300822FFF7B3BF0120704700BF7F
:100B80005C270020014B1868704700BF002004E07C
:100B900070B52A4B1B68C3F30B0204461B0C62B1F1
:100BA00040F21340824230D040F2194082422ED0AF
:100BB00040F2214082422CD10322214D0C2000FB27
:100BC0000252556842F20102934224D0B3F5805F8D
:100BD00023D041F20102934221D041F20302934219
:100BE0001FD041F20702934214BF3F233123013C3F
:100BF0000C44013D0A46A24215D215F9016F501C62
:100C00009EB100F8016C0246F5E70122D5E7022209
:100C1000D3E70C4DD6E73323E9E74123E7E75A232F
:100C2000E5E75923E3E7104605E02C2584421570DB
:100C300001D9901C5370401A70BD00BF002004E021
:100C40003C33000810330008022802BF024B4FF467
:100C500000129A61704700BF00040240022802BFE0
:100C6000014B20229A61704700040240022801BF14
:100C7000024A536983F02003536170470004024025
:100C800010B50023934203D0CC5CC4540133F9E780
:100C900010BD000010B5013810F9013F3BB191F9CA
:100CA00000409C4203D11AB10131013AF4E71AB174
:100CB00091F90020981A10BD1046FCE70346024641
:100CC000D01A12F9011B0029FAD1704702440346D9
:100CD000934202D003F8011BFAE770472DE9F8436D
:100CE0001F4D144695F824200746884652BBDFF86E
:100CF00070909CB395F824302BB92022FF214846F0
:100D00002F62FFF7E3FF95F82400C0F10802A2422A
:100D100028BF2246D6B24146920005EB8000FFF77D
:100D2000AFFF95F82430A41B1E44F6B2082E1744DA
:100D30009044E4B285F82460DBD1FFF713FF00286C
:100D4000D7D108E02B6A03EB82038342CFD0FFF7B1
:100D500009FF0028CBD10020BDE8F8830120FBE784
:100D60005C270020024B1A78024B1A70704700BFB4
:100D7000842700200026002010B50F4C0F4800F0FB
:100D800003F921460D4800F02BF924680C48626DE8
:100D9000D2F8043843F00203C2F8043800F016FE1B
:100DA0000849204600F022FA626DD2F8043823F098
:100DB0000203C2F8043810BD30340008402A002075
:100DC00040420F003834000870470000FEE7000082
:100DD00000B59BB0EFF3098168226846FFF750FF2A
:100DE000EFF30583034B9A6B9A6A9A6A9A6A9A6A36
:100DF0009B6AFEE700ED00E000B59BB0EFF30981D0
:100E000068226846FFF73CFFEFF30583044B9A6BBB
:100E10009A6A9A6A9A6A9A6A9A6A9B6AFEE700BF15
:100E200000ED00E000B59BB0EFF309816822684651
:100E3000FFF726FFEFF30583034B5A6B9A6A9A6A12
:100E40009A6A9A6A9B6AFEE700ED00E030B5094DA8
:100E50000A4491420DD011F8013B5840082340F359
:100E60000004013B2C4013F0FF0384EA5000F6D14C
:100E7000EFE730BD2083B8ED0023054A1946013362
:100E8000102BC2E9001102F10802F8D1704700BF2F
:100E900088270020026843681143016003B11847A6
:100EA0007047000013B5446BD4F894341A68117875
:100EB000042915D1217C022912D119791289012323
:100EC0008B4013420CD101A904F14C0001F084FEC7
:100ED000D4F89444019B21790246206800F0CEF9B1
:100EE00002B010BD143001F007BE00004FF0FF3318
:100EF000143001F001BE00004C3001F0D9BE0000FA
:100F00004FF0FF334C3001F0D3BE0000143001F03D
:100F1000D5BD00004FF0FF31143001F0CFBD00000F
:100F20004C3001F0A5BE00004FF0FF324C3001F014
:100F30009FBE00000020704710B5D0F894341A68A6
:100F400011780429044617D1017C022914D119799A
:100F5000528901238B4013420ED1143001F068FDF9
:100F6000024648B1D4F894444FF480736179206804
:100F7000BDE8104000F070B910BD0000406BFFF7F5
:100F8000DBBF0000704700007FB5124B03600023F9
:100F90004360C0E90233012502260F4B0574044665
:100FA0000290019300F18402294600964FF4807369
:100FB000143001F019FD094B0294CDE9006304F5EA
:100FC00023724FF48073294604F14C0001F0E0FDD8
:100FD00004B070BD6C3300087D0F0008A50E00083A
:100FE0000B68202282F311880A7903EB8202906158
:100FF0004A79093243F822008A7912B103EB82035D
:10100000986102230374C0F89414002383F31188B9
:101010007047000038B5037F044613B190F8543090
:10102000ABB9201D01250221FFF734FF04F11400A4
:1010300025776FF0010100F0F1FC84F8545004F1C1
:101040004C006FF00101BDE8384000F0E7BC38BD4E
:1010500010B5012104460430FFF71CFF002323775D
:1010600084F8543010BD000038B504460025143013
:1010700001F0D2FC04F14C00257701F0A1FD201D08
:1010800084F854500121FFF705FF2046BDE83840A1
:10109000FFF752BF90F8443003F06003202B07D1D4
:1010A00090F84520212A4FF0000303D81F2A06D8C4
:1010B00000207047222AFBD1C0E90E3303E0034A27
:1010C00082630722C2630364012070470126002067
:1010D00037B5D0F894341A681178042904461AD127
:1010E000017C022917D11979128901238B401342FF
:1010F00011D100F14C05284601F022FE58B101A99A
:10110000284601F069FDD4F89444019B21790246F8
:10111000206800F0B3F803B030BD0000F0B500EB7C
:10112000810385B09E6904460D46FEB1202383F3FA
:10113000118804EB8507301D0821FFF7ABFEFB6823
:101140005B691B6806F14C001BB1019001F052FD78
:10115000019803A901F040FD024648B1039B2946CE
:10116000204600F08BF8002383F3118805B0F0BD12
:10117000FB685A691268002AF5D01B8A013B1340AC
:10118000F1D104F14402EAE7093138B550F82140C1
:10119000DCB1202383F31188D4F8942413685279A6
:1011A00003EB8203DB689B695D6845B1042160182D
:1011B000FFF770FE294604F1140001F043FC2046BD
:1011C000FFF7BAFE002383F3118838BD7047000093
:1011D00000F0F4BF012303700023C0E90133C361B1
:1011E00083620362C36243620363704738B5044697
:1011F000202383F311880025C0E90355C0E9055574
:10120000416000F0EBFF0223237085F3118838BDA5
:1012100070B500EB810305465069DA600E4614464E
:1012200018B110220021FFF751FDA06918B110225A
:101230000021FFF74BFD31462846BDE8704001F024
:1012400097B80000826802F0011282600022C0E9B3
:101250000422826101F018B9F0B400EB81044789DF
:10126000E4680125A4698D403D4345812360002346
:10127000A2606360F0BC01F033B90000F0B400EB91
:1012800081040789E468012564698D403D43058137
:1012900023600023A2606360F0BC01F0ADB90000E0
:1012A00070B50223002504460370C0E90255C0E969
:1012B0000455C564856180F8345000F0F5FF63681B
:1012C0001B6823B129462046BDE87040184770BD11
:1012D000027880F850204368052202701B680BB129
:1012E000042118477047000090F8502043680270AE
:1012F0001B680BB1052118477047000070B590F8C6
:101300003430044613B1002380F8343004F1440231
:10131000204601F0DBF863689B68B3B994F8443069
:1013200013F0600535D00021204601F029FB002193
:10133000204601F01BFB63681B6813B106212046A1
:101340009847062384F8343070BD2046984700281B
:10135000E4D0B4F84A30E26B9A4288BFE36394F970
:101360004430E56B002B4FF0200380F20381002D09
:1013700000F0F280092284F8342083F311880021E0
:10138000D4E90E232046FFF779FF002383F3118869
:10139000DAE794F8452003F07F0343EA022340F2A2
:1013A0000232934200F0C58021D8B3F5807F48D047
:1013B0000DD8012B3FD0022B00F09380002BB2D12F
:1013C00004F14C02A2630222E2632364C1E7B3F595
:1013D000817F00F09B80B3F5407FA4D194F8463024
:1013E000012BA0D1B4F84C3043F0020332E0B3F546
:1013F000006F4DD017D8B3F5A06F31D0A3F5C063FF
:10140000012B90D8636894F846205E6894F84710E2
:10141000B4F848302046B047002884D04368A3631E
:101420000368E3631AE0B3F5106F36D040F602426A
:1014300093427FF478AF5C4BA3630223E363002302
:10144000C3E794F84630012B7FF46DAFB4F84C300D
:1014500023F00203C4E90E55A4F84C30256478E764
:10146000B4F84430B3F5A06F0ED194F8463084F848
:101470004E30204600F070FF63681B6813B10121F5
:1014800020469847032323700023C4E90E339CE7CA
:1014900004F14F03A3630123C3E72378042B10D186
:1014A000202383F311882046FFF7CCFE85F31188B3
:1014B0000321636884F84F5021701B680BB12046EC
:1014C000984794F84630002BDED084F84F30042340
:1014D000237063681B68002BD6D0022120469847F2
:1014E000D2E794F848301D0603F00F0120460AD5D4
:1014F00000F0DEFF012804D002287FF414AF2B4B4C
:101500009AE72B4B98E700F0C5FFF3E794F84630D5
:10151000002B7FF408AF94F8483013F00F01B3D0DC
:101520001A06204602D501F03FFAADE701F032FA83
:10153000AAE794F84630002B7FF4F5AE94F84830D3
:1015400013F00F01A0D01B06204602D501F018FAB7
:101550009AE701F00BFA97E7142284F8342083F31A
:1015600011882B462A4629462046FFF775FE85F34B
:101570001188E9E65DB1152284F8342083F31188DF
:101580000021D4E90E232046FFF766FEFDE60B227C
:1015900084F8342083F311882B462A4629462046B6
:1015A000FFF76CFEE3E700BF9C33000894330008AC
:1015B0009833000838B590F834300446002B3ED0FC
:1015C000063BDAB20F2A34D80F2B32D8DFE803F00B
:1015D0003731310822323131313131313131373720
:1015E000C56BB0F84A309D4214D2C3681B8AB5FB64
:1015F000F3F203FB12556DB9202383F311882B46B8
:101600002A462946FFF73AFE85F311880A2384F813
:1016100034300EE0142384F83430202383F311880F
:1016200000231A4619462046FFF716FE002383F3CF
:10163000118838BD036C03B198470023E7E7002108
:10164000204601F09DF90021204601F08FF96368E2
:101650001B6813B10621204698470623D7E70000F0
:1016600010B590F83430142B044629D017D8062B27
:1016700005D001D81BB110BD093B022BFBD80021BE
:10168000204601F07DF90021204601F06FF96368E2
:101690001B6813B1062120469847062319E0152B35
:1016A000E9D10B2380F83430202383F31188002301
:1016B0001A461946FFF7E2FD002383F31188DAE7A3
:1016C000C3689B695B68002BD5D1036C03B1984755
:1016D000002384F83430CEE7024B0022C3E9003304
:1016E0009A60704708280020002303748268054B25
:1016F0001B6899689142FBD25A680360426010608F
:10170000586070470828002008B5202383F311880B
:10171000037C032B05D0042B0DD02BB983F3118848
:1017200008BD436900221A604FF0FF334361FFF7A1
:10173000DBFF0023F2E7D0E9003213605A60F3E7E1
:10174000002303748268054B1B6899689142FBD89B
:101750005A68036042601060586070470828002093
:10176000054B19690874186802681A60536018619B
:1017700001230374FEF7C8BD0828002030B54B1CB8
:101780000B4D87B0044610D02B690A4A01A800F01F
:1017900061F92046FFF7E4FF049B13B101A800F0B4
:1017A00093F92B69586907B030BDFFF7D9FFF8E707
:1017B000082800200917000838B50C4D41612B6935
:1017C00081689A689142044603D8BDE83840FFF723
:1017D0008BBF1846FFF788FF01232C610146237455
:1017E0002046BDE83840FEF78FBD00BF0828002026
:1017F000044B1A681B6990689B68984294BF00204C
:10180000012070470828002010B5084C2368206983
:101810001A6822605460012223611A74FFF790FF56
:1018200001462069BDE81040FEF76EBD0828002083
:10183000FFF7EABFFEE7000010B5184CFFF74CFFBA
:1018400000F0FAF816498022204600F081F80123C2
:1018500044F8180C0374134B134AD96821F4E0615F
:101860000904090C0A43DA60D3F8FC200F4942F05E
:101870008072C3F8FC200A6842F001020A6010225C
:10188000DA77202283F82220002383F3118862B6BE
:101890000748BDE8104000F07BB800BF30280020AA
:1018A000A033000800ED00E00003FA05001000E09E
:1018B000B03300082DE9F0471F4D2E464FF00008C9
:1018C00056F8144FA2684FF08043586A2B6AC71A23
:1018D00097421DD34FF02009A2682B6AD4F80CA0C0
:1018E00013442B622368B3425E60A7EB02076B616F
:1018F000C4F80C8001D101F04BFA88F311882069FB
:10190000D04789F311886C69A3689F42E4D2D9E774
:101910006A69B2420DD0916828620B441B1A936029
:10192000A368BDE8F047022B2CBFC018023001F0BD
:1019300035BABDE8F08700BF08280020034A516887
:1019400053685B1A9842FBD8704700BF001000E054
:1019500082600222028270478368A3F17C0243F80E
:101960000C2C026943F83C2C426943F8382C074A96
:1019700043F81C2CC26843F8102C022203F8082CF0
:10198000002203F8072CA3F1180070472103000878
:1019900010B5202383F31188FFF7DEFF00210446F2
:1019A000FFF70AFF002383F31188204610BD0000D3
:1019B000024B1B6958610F20FFF7D2BE0828002098
:1019C000202383F31188FFF7F3BF000008B5014619
:1019D000202383F311880820FFF7D0FE002383F330
:1019E000118808BD49B1064B42681B6918605A60EE
:1019F000136043600420FFF7C1BE4FF0FF30704713
:101A0000082800200368984206D01A6802605060D7
:101A100059611846FFF768BE7047000038B50446A4
:101A20000D462068844200D138BD036823605C60A5
:101A30004561FFF759FEF4E7054B03F11402C3E9D2
:101A400005224FF0FF310022C3E90712704700BFA3
:101A500008280020F8B5C0E903231A4F4FF080434F
:101A600002295C6A3B4638BF022153F8145F9D424D
:101A700006460AD1C7E905003C62C0E9005581600D
:101A80000819BDE8F84001F07BB9386AAB68241A40
:101A90000C1902D32D68E41A04E0A34202D92044B1
:101AA00001F07CF9AB68A342F4D36B6873603560D6
:101AB0001E606E60B460AB681B1BAB604FF0FF3301
:101AC000FB61F8BD08280020184903680A4630B4B5
:101AD00052F8144F84424FF000050BD041689342F6
:101AE0000B605960C56003D09A6881680A449A60A7
:101AF00030BC704793424B615A60E56002D130BC04
:101B000001F046B99A68A06802449A604FF0804399
:101B1000086A5B6A191A8A42EAD9C31A1344012B6C
:101B200098BF8A1C30BC104401F038B90828002046
:101B300000207047FEE70000704700004FF0FF30C4
:101B40007047000002290CD0032904D0012907485E
:101B500018BF00207047032A05D8054800EBC200D3
:101B60007047044870470020704700BF9434000855
:101B7000082600204834000870B59AB0054608468B
:101B800001A9144600F098F801A8FFF797F8431C44
:101B90005B00C5E900340022237003236370C6B2E2
:101BA00001AB02341046D1B28E4204F1020401D8D6
:101BB0001AB070BD13F8011B04F8021C04F8010CE4
:101BC0000132F0E708B5202383F311880348FFF7BB
:101BD0007FFA002383F3118808BD00BF402A00204C
:101BE00007B5052917D8DFE801F0191603191920E0
:101BF000202383F31188104A01900121FFF708FB8D
:101C000001980E4A0221FFF703FB0D48FFF72CFA5B
:101C1000002383F3118803B05DF804FB202383F3D2
:101C200011880748FFF7F6F9F2E7202383F31188BC
:101C30000348FFF70DFAEBE7E83300080C3400081F
:101C4000402A002038B50C4D0C4C0D492A4604F1B1
:101C50000800FFF791FF05F1CA0204F110000949DD
:101C6000FFF78AFF05F5CA7204F118000649BDE8BE
:101C70003840FFF781BF00BF082F00200826002052
:101C8000C8330008D2330008DD33000870B50446BD
:101C900008460D46FFF712F8C6B220460134037815
:101CA0000BB9184670BD32462946FEF7F3FF0028EF
:101CB000F3D10120F6E700002DE9F84F05460C4668
:101CC000FEF7FCFF2B49C6B22846FFF7DFFF08B13D
:101CD0000436F6B228492846FFF7D8FF08B1103677
:101CE000F6B2632E0DD8DFF88C90DFF88CA0DFF809
:101CF0009480DFF894B0214F2E7846B92670BDE865
:101D0000F88F29462046BDE8F84F01F0F9BA252E94
:101D10002CD1072249462846FEF7BCFF50B93B6844
:101D200023607B6863603B892381BB7AA37207359C
:101D30000B34E1E7082251462846FEF7ABFFA8B96D
:101D40000F4BA21C19780909023211F8081002F889
:101D5000041C13F8011B01F00F015B4511F808107A
:101D600002F8031CEED118340835C5E704F8016BFE
:101D70000135C1E7B4340008DD330008BC34000885
:101D8000107AFF1FC83400081C7AFF1FBFF34F8F63
:101D9000024AD368DB03FCD4704700BF003C02401A
:101DA00008B5094B1B7873B9FFF7F0FF074B1A69A9
:101DB000002ABFBF064A5A6002F188325A601A6888
:101DC00022F480621A6008BD66310020003C0240A7
:101DD0002301674508B50B4B1B7893B9FFF7D6FF76
:101DE000094B1A6942F000421A611A6842F48052A3
:101DF0001A601A6822F480521A601A6842F48062EB
:101E00001A6008BD66310020003C02400B28F0B586
:101E100016D80C4C0C4923787BB90C4D0E460C237C
:101E20004FF0006255F8047B46F8042B013B13F099
:101E3000FF033A44F6D10123237051F82000F0BD8E
:101E40000020FCE79831002068310020DC340008D5
:101E5000014B53F820007047DC3400080C20704719
:101E60000B2810B5044601D9002010BDFFF7CEFFA6
:101E7000064B53F824301844C21A0BB90120F4E77A
:101E800012680132F0D1043BF6E700BFDC340008F1
:101E90000B2810B5044621D8FFF778FFFFF780FF25
:101EA0000F4AF323D360C300DBB243F4007343F063
:101EB00002031361136943F480331361FFF766FF74
:101EC000FFF7A4FF074B53F8241000F0D9F8FFF7F1
:101ED00081FF2046BDE81040FFF7C2BF002010BDC3
:101EE000003C0240DC340008F8B512F0010314464F
:101EF00042D18218B2F1016F57D22D4B1B6813F0FB
:101F0000010352D02B4DFFF74BFFF323EB60FFF79C
:101F10003DFF40F20127032C15D824F00104661878
:101F2000244C401A40F20117B142236900EB01052D
:101F300024D123F001032361FFF74CFF0120F8BDFA
:101F4000043C0430E7E78307E7D12B6923F44073AF
:101F50002B612B693B432B6151F8046B0660BFF387
:101F60004F8FFFF713FF03689E42E9D02B6923F0E0
:101F700001032B61FFF72EFF0020E0E723F44073FD
:101F8000236123693B4323610B882B80BFF34F8F71
:101F9000FFF7FCFE2D8831F8023BADB2AB42C3D057
:101FA000236923F001032361E4E71846C7E700BF74
:101FB00000380240003C0240084908B50B7828B1BF
:101FC0001BB9FFF7EDFE01230B7008BD002BFCD001
:101FD000BDE808400870FFF7FDBE00BF6631002075
:101FE00010B50244064BD2B2904200D110BD441C41
:101FF00000B253F8200041F8040BE0B2F4E700BF50
:10200000502800400F4B30B51C6F240407D41C6FC0
:1020100044F400741C671C6F44F400441C670A4CB1
:10202000236843F4807323600244084BD2B2904289
:1020300000D130BD441C00B251F8045B43F820507D
:10204000E0B2F4E700380240007000405028004041
:1020500007B5012201A90020FFF7C2FF019803B0D4
:102060005DF804FB13B50446FFF7F2FFA04205D06C
:10207000012201A900200194FFF7C4FF02B010BDA6
:1020800070470000044BD3F874389B0042BF034BE9
:1020900001221A70704700BF0030024099310020C1
:1020A000014B1878704700BF99310020704700003D
:1020B000FEE700000A4B0B480B4A90420BD30B4B38
:1020C000DA1C121AC11E22F003028B4238BF002212
:1020D0000021FEF7FBBD53F8041B40F8041BECE79E
:1020E0006036000814320020143200201432002020
:1020F00030B5D0E9154300229D6811464FF0FF30FE
:1021000004EB421301329542C3F80019C3F81019C9
:10211000C3F80809C3F8001BC3F8101BC3F8080B69
:10212000EED24FF00113C4F81C3830BD1D4B03EB49
:1021300080022DE9F043D2F80CC05D6DDCF814206C
:10214000461CD2F800E005EB063605EB4018516856
:1021500071450AD3D5F83438012202FA00F023EA97
:102160000000C5F83408BDE8F083BCF81040AEEBC1
:102170000103A34228BF2346D8F81849A4B2B3EB01
:10218000840FF0D89468A4F1040959F8047F3760EB
:10219000A4EB09071F44042FF7D81C440B44946098
:1021A0005360D4E79C310020890141F02001016196
:1021B00003699B06FCD41220FFF7C0BB10B5054C89
:1021C0002046FFF707F84FF0A0436365024BA36575
:1021D00010BD00BF9C3100203035000870B5037879
:1021E000012B054650D12A4B446D98421BD1294BF7
:1021F0005A6B42F080025A635A6D42F080025A656F
:102200005A6D5A6942F080025A615A6922F080027E
:102210005A610E2143205B6900F0D0FB1E4BE36046
:102220001E4BC4F800380023C4F8003EC0232360CE
:102230006E6D4FF40413A3633369002BFCDA0123A2
:1022400033610C20FFF77AFB3369DB07FCD41220E3
:10225000FFF774FB3369002BFCDA0026A6602846E2
:10226000FFF746FF6B68C4F81068DB68C4F81468B1
:10227000C4F81C684BB90A4BA3614FF0FF3363618C
:10228000A36843F00103A36070BD064BF4E700BFF1
:102290009C3100200038024040140040030020021E
:1022A000003C30C0083C30C0F8B5446D0546002104
:1022B0002046FFF779FFA96D00234FF001128F68C8
:1022C000C4F834384FF00066C4F81C284FF0FF30D3
:1022D00004EB431201339F42C2F80069C2F8006B5D
:1022E000C2F80809C2F8080BF2D20B686A6DEB65F8
:1022F000636210231361166916F01006FBD11220D9
:10230000FFF71CFBD4F8003823F4FE63C4F8003850
:10231000A36943F4402343F01003A3610923C4F8E5
:102320001038C4F814380A4BEB604FF0C043C4F8BF
:10233000103B084BC4F8003BC4F81069C4F80039DE
:10234000EB6D03F1100243F48013EA65A362F8BD5C
:102350000C35000840800010426D90F84E10D2F805
:10236000003823F4FE6343EA0113C2F800387047D3
:102370002DE9F84300EB8103456DDA68166806F035
:102380000306731E022B05EB41130C4680460FFA21
:1023900081F94FEA41104FF00001C3F8101B4FF0D4
:1023A000010104F1100398BFB60401FA03F3916927
:1023B0008EBF334E06F1805606F5004600293AD00E
:1023C000578A04F15801490137436F50D5F81C185A
:1023D0000B43C5F81C382B180021C3F8101953699A
:1023E0000127611EA7409BB3138A928B9B08012A89
:1023F00088BF5343D8F85C20981842EA034301F1A0
:10240000400205EB8202C8F85C0021465360284672
:10241000FFF7CAFE08EB8900C3681B8A43EA8453AE
:10242000483464011E432E51D5F81C381F43C5F8AB
:102430001C78BDE8F88305EB4917D7F8001B21F499
:102440000041C7F8001BD5F81C1821EA0303C0E7B8
:1024500004F13F0305EB83030A4A5A6028462146EC
:10246000FFF7A2FE05EB4910D0F8003923F4004332
:10247000C0F80039D5F81C3823EA0707D7E700BFB2
:102480000080001000040002826D1268C265FFF730
:102490002FBE00005831436D49015B5813F40040D2
:1024A00004D013F4001F0CBF02200120704700006D
:1024B0004831436D49015B5813F4004004D013F4D4
:1024C000001F0CBF022001207047000000EB8101BB
:1024D000CB68196A0B6813604B6853607047000043
:1024E00000EB810330B5DD68AA691368D36019B9C0
:1024F000402B84BF402313606B8A1468426D1C44D8
:10250000013CB4FBF3F46343033323F0030302EB16
:10251000411043EAC44343F0C043C0F8103B2B686A
:1025200003F00303012B09B20ED1D2F8083802EBF5
:10253000411013F4807FD0F8003B14BF43F0805368
:1025400043F00053C0F8003B02EB4112D2F8003BCD
:1025500043F00443C2F8003B30BD00002DE9F041D8
:10256000244D6E6D06EB40130446D3F8087BC3F888
:10257000087B38070AD5D6F81438190706D505EBB5
:1025800084032146DB6828465B689847FA071FD515
:10259000D6F81438DB071BD505EB8403D968CCB912
:1025A0008B69488A5A68B2FBF0F600FB16228AB99A
:1025B0001868DA6890420DD2121AC3E90024202369
:1025C00083F311880B482146FFF78AFF84F31188B3
:1025D000BDE8F081012303FA04F26B8923EA0203C8
:1025E0006B81CB68002BF3D021460248BDE8F04157
:1025F000184700BF9C31002000EB810370B5DD68F7
:10260000436D6C692668E6604A0156BB1A444FF474
:102610000020C2F810092A6802F00302012A0AB257
:102620000ED1D3F8080803EB421410F4807FD4F8DD
:10263000000914BF40F0805040F00050C4F8000979
:1026400003EB4212D2F8000940F00440C2F800093E
:10265000D3F83408012202FA01F10143C3F8341817
:1026600070BD19B9402E84BF4020206020682E8A9A
:102670008419013CB4FBF6F440EAC44040F0005039
:102680001A44C6E7F8B504461E48456D05EB4413E9
:10269000D3F80869C3F80869F10717D5D5F81038D9
:1026A000DA0713D500EB8403D9684B691F68DA6831
:1026B000974218D2D21B00271A605F60202383F351
:1026C00011882146FFF798FF87F31188330617D545
:1026D000D5F834280123A340134211D02046BDE889
:1026E000F840FFF723BD012303FA04F2038923EA2C
:1026F000020303818B68002BE8D021469847E5E769
:10270000F8BD00BF9C3100202DE9F74F964C666D57
:102710007569B3691D4015F48058756107D020466E
:10272000FEF7BEFD03B0BDE8F04F00F0BDBB002DCD
:1027300012DAD6F8003E8C489F071EBFD6F8003E3E
:1027400023F00303C6F8003ED6F8043823F0010353
:10275000C6F80438FEF7C8FD280502D58248FEF702
:10276000B7FDA9040CD5D6F8083813F0060FF368A6
:1027700023F470530CBF43F4105343F4A053F3609D
:102780002A0704D56368DB680BB177489847EB02EA
:1027900074D4AF0227D5D4F85490DFF8CCB1002719
:1027A0004FF0010A09EB4712D2F8003B03F4402333
:1027B000B3F5802F11D1D2F8003B002B0DDA6289DE
:1027C0000AFA07F322EA0303638104EB8703DB6859
:1027D000DB6813B1394658469847A36D01379B68AB
:1027E000FFB29F42DED9E80617D5676D3A6AC2F399
:1027F0000A1002F00F0302F4F012B2F5802F00F07D
:102800008880B2F5402F08D104EB83030022DB68F7
:102810001B6A07F5805790426DD12903D6F81848F6
:1028200013D5E20302D50020FFF798FEA30302D5DB
:102830000120FFF793FE670302D50220FFF78EFE0B
:10284000260302D50320FFF789FE6D037FF56AAFEB
:10285000E00702D50020FFF715FFA10702D50120F0
:10286000FFF710FF620702D50220FFF70BFF2307D7
:102870007FF558AF0320FFF705FF53E7636DDFF8DF
:10288000E8B0019300274FF0010AA36D9B685FFA3F
:1028900087F999453FF67DAF019B03EB4913D3F8C8
:1028A000002902F44022B2F5802F22D1D3F800296A
:1028B000002A1EDAD3F8002942F09042C3F800291A
:1028C000D3F80029002AFBDB606D4946FFF76CFC5A
:1028D00022890AFA09F322EA0303238104EB89031C
:1028E000DB689B6813B14946584698474846FFF74E
:1028F0001DFC0137C9E7910708BFD7F80080072AF8
:1029000098BF03F8018B02F1010298BF4FEA182823
:1029100081E7023304EB830207F580575268D2F84F
:1029200018C0DCF80820DCE9001CA1EB0C0C00212D
:1029300088420AD104EB830463689B699A68024465
:102940009A605A6802445A6067E711F0030F08BFA3
:10295000D7F800808C4588BF02F8018B01F1010196
:1029600088BF4FEA1828E3E79C310020436D03EB52
:102970004111D1F8003B43F40013C1F8003B70470C
:10298000436D03EB4111D1F8003943F40013C1F852
:1029900000397047436D03EB4111D1F8003B23F43C
:1029A0000013C1F8003B7047436D03EB4111D1F8B0
:1029B000003923F40013C1F80039704700F1604377
:1029C00003F561430901C9B283F80013012200F045
:1029D0001F039A4043099B0003F1604303F56143E1
:1029E000C3F880211A60704730B5039C017204332C
:1029F00004FB0325C0E90653049B03630021059BE8
:102A0000C160C0E90000C0E90422C0E90842C0E991
:102A10000A11436330BD0000416A0022C0E904117D
:102A2000C0E90A22C2606FF00101FEF7F7BF0000A3
:102A3000D0E90432934201D1C2680AB9181D704727
:102A40000020704703691960C2680132C260C26920
:102A5000134482690361934224BF436A03610021E6
:102A6000FEF7D0BF38B504460D46E3683BB1626956
:102A7000131D1268A3621344E362002007E0237A67
:102A800033B929462046FEF7ADFF0028EDDA38BD00
:102A90006FF00100FBE70000C368C269013BC3603F
:102AA0004369134482694361934224BF436A43618B
:102AB00000238362036B03B11847704770B520236E
:102AC000044683F31188866A3EB9FFF7CBFF0546BB
:102AD00018B186F31188284670BDA36AE26A13F81C
:102AE000015BA362934202D32046FFF7D5FF002388
:102AF00083F31188EFE700002DE9F84F04460E46F6
:102B0000174698464FF0200989F311880025AA46F8
:102B1000D4F828B0BBF1000F09D141462046FFF799
:102B2000A1FF20B18BF311882846BDE8F88FD4E9C6
:102B30000A12A7EB050B521A934528BF9346BBF127
:102B4000400F1BD9334601F1400251F8040B43F802
:102B5000040B9142F9D1A36A40334036A362403559
:102B6000D4E90A239A4202D32046FFF795FF8AF35D
:102B70001188BD42D8D289F31188C9E730465A4638
:102B8000FEF77EF8A36A5B445E44A3625D44E7E718
:102B900010B5029C0172043304FB0321C0E9061343
:102BA0000023C0E90A33039B0363049BC460C0E9AC
:102BB0000000C0E90422C0E90842436310BD0000E0
:102BC000026AC260426AC0E904220022C0E90A2205
:102BD0006FF00101FEF722BFD0E904239A4201D130
:102BE000C26822B9184650F8043B0B6070470020B9
:102BF00070470000C368C2690133C360436913446E
:102C000082694361934224BF436A43610021FEF716
:102C1000F9BE000038B504460D46E3683BB12369B0
:102C20001A1DA262E2691344E362002007E0237ADE
:102C300033B929462046FEF7D5FE0028EDDA38BD27
:102C40006FF00100FBE7000003691960C268013AF8
:102C5000C260C269134482690361934224BF436A1C
:102C6000036100238362036B03B1184770470000C0
:102C700070B520230D460446114683F31188866AF9
:102C80002EB9FFF7C7FF10B186F3118870BDA36A94
:102C90001D70A36AE26A01339342A36204D3E1691F
:102CA00020460439FFF7D0FF002080F31188EDE7BC
:102CB0002DE9F84F04460D46904699464FF0200AFC
:102CC0008AF311880026B346A76A4FB949462046C1
:102CD000FFF7A0FF20B187F311883046BDE8F88FD9
:102CE000D4E90A073A1AA8EB0607974228BF174605
:102CF000402F1BD905F1400355F8042B40F8042B55
:102D00009D42F9D1A36A4033A3624036D4E90A2335
:102D10009A4204D3E16920460439FFF795FF8BF30B
:102D200011884645D9D28AF31188CDE729463A461B
:102D3000FDF7A6FFA36A3B443D44A3623E44E5E79A
:102D4000D0E904239A4217D1C3689BB1836A8BB13F
:102D5000043B9B1A0ED01360C368013BC360C36978
:102D60001A44836902619A4224BF436A03610023C3
:102D700083620123184670470023FBE700F0D6B8B2
:102D80004FF08043002258631A610222DA607047D4
:102D90004FF080430022DA60704700004FF080431C
:102DA000586370474B6843608B688360CB68C3602F
:102DB0000B6943614B6903628B6943620B68036073
:102DC0007047000008B5264B26481A6940F2FF11EB
:102DD0000A431A611A6922F4FF7222F001021A6191
:102DE0001A691A6B0A431A631A6D0A431A651E4A56
:102DF0001B6D1146FFF7D6FF02F11C0100F5806044
:102E0000FFF7D0FF02F1380100F58060FFF7CAFF3D
:102E100002F1540100F58060FFF7C4FF02F1700178
:102E200000F58060FFF7BEFF02F18C0100F58060C5
:102E3000FFF7B8FF02F1A80100F58060FFF7B2FFCD
:102E400002F1C40100F58060FFF7ACFF02F1E00180
:102E500000F58060FFF7A6FFBDE8084000F0D0B89D
:102E600000380240000002403C35000808B500F080
:102E700037FAFEF7E1FCFFF705F9BDE80840FEF779
:102E8000E1BE000070470000064A536B23F00103C7
:102E90005363EFF30983683383F30988002383F3D3
:102EA0001188704700EF00E010B5202383F31188EC
:102EB000104B5B6813F4006318D0F1EE103AEFF397
:102EC00009844FF0807344F84C3C0B4BDB6B44F8A7
:102ED000083CA4F1680383F30988FEF789FC18B164
:102EE000064B44F8503C10BD054BFAE783F31188BC
:102EF000F9E700BF00ED00E000EF00E0310300085B
:102F0000340300084FF0804310B51A69920708D5C2
:102F100000241C61202383F31188FEF7CBFC84F38B
:102F20001188BDE81040FFF7BFBF0000104B1A6CBE
:102F300042F001021A641A6E42F001021A660D4A4A
:102F40001B6E936843F0010393604FF0804353225C
:102F50009A624FF0FF32DA6200229A615A63DA60B5
:102F60005A6001225A6108211A601C20FFF726BD11
:102F700000380240002004E01F4B1A696FEAC25279
:102F80006FEAD2521A611A69C2F308021A614FF04D
:102F9000FF301A695A69586100215A6959615A69A2
:102FA0001A6A62F080521A621A6A02F080521A6239
:102FB0001A6A5A6A58625A6A59625A6A1A6C42F014
:102FC00080521A641A6E42F080521A661A6E0B4AC8
:102FD000106840F480701060186F00F44070B0F515
:102FE000007F1EBF4FF4803018671967536823F4C1
:102FF0000073536000F054B9003802400070004084
:10300000304B4FF080521A642F4A4FF44041116008
:103010001A6842F001021A601A689107FCD59A6892
:1030200022F003029A60274B9A6812F00C02FBD13F
:10303000196801F0F90119609A601A6842F4803247
:103040001A601A689203FCD55A6F42F001025A675F
:103050001C4B5A6F9007FCD51C4A5A601A6842F004
:1030600080721A60184A53685904FCD5154B1A68C7
:103070009201FCD5164A9A60164B1A68164B9A4272
:10308000164B1BD1164A1168164A914216D140F2CE
:1030900005121A600B4B9A6842F002029A609A6815
:1030A00002F00C02082AFAD15A6C42F480425A64A7
:1030B0005A6E42F480425A665B6E704740F2057267
:1030C000E7E700BF003802400070004008544007A6
:1030D00000948838002004E011640020003C024085
:1030E00000ED00E041C20F41084A08B5516913687C
:1030F0000B4003F00103536123B1054A13680BB180
:1031000050689847BDE80840FFF7CEBE003C01403C
:1031100088270020084A08B5516913680B4003F05E
:103120000203536123B1054A93680BB1D0689847F5
:10313000BDE80840FFF7B8BE003C014088270020EA
:10314000084A08B5516913680B4003F00403536142
:1031500023B1054A13690BB150699847BDE808408F
:10316000FFF7A2BE003C014088270020084A08B5AE
:10317000516913680B4003F00803536123B1054AFA
:1031800093690BB1D0699847BDE80840FFF78CBE42
:10319000003C014088270020084A08B5516913689F
:1031A0000B4003F01003536123B1054A136A0BB1BE
:1031B000506A9847BDE80840FFF776BE003C0140E2
:1031C00088270020174B10B55A691C68144004F476
:1031D00078725A61A30604D5134A936A0BB1D06A78
:1031E0009847600604D5104A136B0BB1506B984793
:1031F000210604D50C4A936B0BB1D06B9847E205BE
:1032000004D5094A136C0BB1506C9847A30504D53B
:10321000054A936C0BB1D06C9847BDE81040FFF79E
:1032200043BE00BF003C0140882700201A4B10B568
:103230005A691C68144004F47C425A61620504D542
:10324000164A136D0BB1506D9847230504D5134AE8
:10325000936D0BB1D06D9847E00404D50F4A136EFF
:103260000BB1506E9847A10404D50C4A936E0BB174
:10327000D06E9847620404D5084A136F0BB1506FA3
:103280009847230404D5054A936F0BB1D06F984734
:10329000BDE81040FFF708BE003C01408827002031
:1032A000062108B50846FFF789FB06210720FFF72E
:1032B00085FB06210820FFF781FB06210920FFF787
:1032C0007DFB06210A20FFF779FB06211720FFF777
:1032D00075FBBDE8084006212820FFF76FBB000002
:1032E00008B5FFF749FEFDF7C7FDFDF771FFFDF7D4
:1032F00049FEFFF7C7FDBDE80840FFF73FBD0000EE
:10330000034611F8012B03F8012B002AF9D170476D
:1033100053544D3332463F3F3F00000053544D332A
:1033200032463430780053544D33324634327800CC
:1033300053544D33324634343658580000000000A0
:10334000103300083F000000130400001C33000885
:103350003F00000019040000263300083F00000071
:1033600021040000303300083F000000000000008E
:10337000010F0008ED0E0008290F0008150F0008C6
:10338000210F00080D0F0008F90E0008E50E0008D7
:10339000350F0008000000000100000000000000E0
:1033A0006D61696E0000000069646C6500000000DA
:1033B000A833000848280020402A0020010000000F
:1033C00035180008000000004172647550696C6F88
:1033D000740025424F415244252D424C002553454F
:1033E0005249414C2500000002000000000000008E
:1033F0001D1100088911000840004000D82E00204F
:10340000E82E002002000000000000000300000081
:1034100000000000CD1100080000000010000000B6
:10342000F82E002000000000010000000000000055
:103430009C31002001010200E11B0008451B00082F
:1034400095100008C51B0008430000005034000818
:1034500009024300020100C0320904000001020217
:1034600001000524001001052401000104240202CA
:103470000524060001070582030800FF0904010076
:10348000020A000000070501024000000705810252
:1034900040000000120000009C34000812011001DE
:1034A000020000400912415700020102030100001E
:1034B0000403090425424F41524425004D616D62C9
:1034C0006146343035763200303132333435363778
:1034D00038394142434445460000000000400000A6
:1034E000004000000040000000400000000001001B
:1034F00000000200000002000000020000000200C4
:1035000000000200000002000000020000000000B5
:10351000FD120008B51500086116000840004000C3
:10352000FC310020FC310020010000000C320020A2
:103530008000000040010000030000000000800245
:1035400000000000AAAAAAAA00000000FFFF0000D5
:103550000000000000A00A000005000000000000BC
:10356000AAAAAAAA00000000CFFF000000000000E5
:10357000000000000000000000000000AAAAAAAAA3
:1035800000000000FFFF000000000000000000003D
:103590000000000000000000AAAAAAAA0000000083
:1035A000FFFF00000000000000000000000000001D
:1035B00000000000AAAAAAAA00000000FFFF000065
:1035C00000000000000000000000000000000000FB
:1035D000AAAAAAAA00000000FFFF00000000000045
:1035E000000000000000000000000000AAAAAAAA33
:1035F00000000000FFFF00000000000000000000CD
:1036000000000000000000000A00000000000000B0
:1036100003000000000000000000000000000000A7
:10362000000000000000000000000000000000009A
:103630000000000000000000FF00960000000008ED
:1036400004000000B034000800000000000000008A
:10365000000000000000000000000000000000006A
:00000001FF
